:020000040000FA
:0A00000020280000000000006A281C
:10004000640003138316053081008312A0308B00F7
:1000500083168C01831608308E00831285010730C9
:100060009F00831620308500831286018316860147
:100070008312B5308100A001A101A20183169B016A
:100080001C141A088312A30083169B0A1C141A0856
:100090008312A40083169B0A1C141A088312A5005D
:1000A00083169B0A1C141A088312A6007D30AB002D
:1000B000A701851E5928A8142708FC3E0319FB3008
:1000C000053EA700A8186228851A6428A814A81855
:1000D00067285928A9000308AA00B53081000B1130
:1000E000A00A2008053C031D8528A001A801831251
:1000F000A10A21082B3C031D8528A100270882079F
:100100009028FA28F228EB28E42820088207022900
:1001100007290C29112916292A0883002908090012
:10012000A20A22083C3C031D8528A200A30A23083A
:100130003C3C031DB028A300A40A2408183C031D5E
:10014000B028A400A50A2508203C031DB0280130D2
:10015000A500A60A26080D3C031DB0280130A60004
:1001600083161C159B018312230883169A005530B1
:100170009D00AA309D009C149C18BB289B0A8312EA
:10018000240883169A0055309D00AA309D009C14C7
:100190009C18C7289B0A8312250883169A0055309D
:1001A0009D00AA309D009C149C18D3289B0A8312A2
:1001B000260883169A0055309D00AA309D009C1495
:1001C0009C18DF2883128528A30A23083C3C031DC2
:1001D0008528A3008528A40A2408183C031D852827
:1001E000A4008528A50A2508203C031D8528013088
:1001F000A5008528A60A26080D3C031D8528013088
:10020000A60085281E308500220886008C281D3017
:100210008500230886008C281B3085002408860072
:100220008C2817308500250886008C280F30850023
:06023000260886008C2860
:02400E00F83F79
:0842000000000C000B000B0094
:00000001FF
